:03000000020027D4
:04000B001204183291
:100023001204AA3275901F75B0CB53D0E775810FB8
:10003300C2AFC28CC28EC23F7589217598D05387D7
:1000430000758C00758A00758DFD758BFDD28E75DC
:10005300B810D2AFD2A91202F012042DD2AC1203FF
:10006300541203952093FD1202F075580075590040
:10007300755A00755B002092031200E430930B3035
:10008300921330911B30902380F21200B93093FD0C
:100093001203F380E71201683092FD1203F380DC50
:1000A3001201E73091FD1203F380D112021F309049
:1000B300FD1203F380C61202F012035412039512C9
:1000C30002533093FD1203F31202F0755800755971
:1000D30000755A00755B001202651203161201685F
:1000E300223092FD1203F33093FD1203F37D0012CD
:1000F300029B12031630905030912F3092053093AB
:100103001980F21203F30DBD04027D0012029B124B
:1001130003163092FD1203F380DB1203F312026520
:100123001203163093FD1203F3221203F3C3ED24DB
:1001330058F8E614B4FF027409F612029B12031670
:100143003091FD1203F380AD1203F3C3ED2458F88D
:10015300E604B40A01E4F612029B1203163090FD82
:100163001203F38090D2B212040779387A047541EE
:10017300007406D29BF5993099FDC299C29B75997B
:10018300053099FDC299E709F5996541F541309923
:10019300FDC299DAF18541993099FDC2991203FDA7
:1001A300C2B2309401221201DAC233780079607A44
:1001B3000808E7600AD233120368303502A74509FD
:1001C300DAEF79601203AB2094073093042033D91C
:1001D3002274FF12047922785079607A08E6F708CE
:1001E30009DAFA22C3E5589401B4FF027409B3F59E
:1001F30058E5599400B4FF027409B3F559E55A94CC
:1002030000B4FF027409B3F55AE55B9400B4FF022E
:100213007409B3F55B12026512031622C3E5582471
:1002230001B40A01E4B3F558E5593400B40A01E412
:10023300B3F559E55A3400B40A01E4B3F55AE55B62
:100243003400B40A01E4B3F55B120265120316220B
:100253007548FF7547FF0000000000D547F8D548F3
:10026300F522C2347938E55B60042410D2342420AB
:10027300F709E55A20340260042410D2342420F70D
:1002830009E55920340260042410D2342420F709EC
:10029300E55824102420F722C2347938E55B600343
:1002A3000202A9BD03042410D2342420F709E55A1D
:1002B30060030202BE203403BD02042410D234249E
:1002C30020F709E55960030202D3203403BD01047A
:1002D3002410D2342420F709E55860030202E820F1
:1002E3003403BD00042410D2342420F722C2B5C243
:1002F300B4C2B37A027928D2B400D2B500C2B50031
:10030300C2B400D2B500C2B500D9F8DAE874FF125E
:10031300047922C2B39004C078387A04D2B400D2EC
:10032300B500C2B500E6C3942093A23792E07908E2
:100333003392B400D2B500C2B500D9F408DAE6E6C8
:1003430054C079063392B400D2B500C2B500D9F4D3
:1003530022780079507A0808120368E4A235340041
:10036300F709DAF322D235E81203C275483C754720
:1003730022203B08D547FAD548F7C235C23B75481A
:100383003C754722203B08D547FAD548F7C235C20A
:100393003B2275385075394F753A4C753B4CC23713
:1003A300711679501203AB227A08E4F5F0C3E71310
:1003B300C5F033C5F009DAF6C5F0F412047922D298
:1003C300B21204072450C4D29BF5993099FDC29907
:1003D300C29B7599023099FDC2997599013099FDB7
:1003E300C2997599013099FDC299C2B21203FD22D7
:1003F300754A0575499A12041122754A0175491007
:1004030012041122754A0175499A12041122D54921
:10041300FDD54AFA2230390BDB08B23771167B0857
:10042300D23622C28CC2377116227B08C236D23929
:10043300D28CD2D37A007C1A90048D7B047838A9AD
:100443000AE993F60809DBF9C2D310360280FBD21E
:10045300D30ADCE474FFC3780813C0E0120479C242
:10046300D310360280FBD2D3D0E0D3D8EC51F0C204
:10047300D3C28CC23922C295C2977908339296D2DD
:1004830095C295D9F7D297C29722202020205345B1
:100493004C4620744553742030313233343536376B
:1004A3003839204C45645320980122C0E0C0D0D293
:1004B300D3D23B859945D0D0D0E0C29822000044E6
:1004C30000000000409CF0000004020000FC60DA21
:1004D300F266B6BEE0FEF60000000000CA00EEFEC3
:1004E3009CFC9E8EBC6E60F8001C0000FCCE0000DD
:1004F300B6007C00000000009D00F0001004FA3EEE
:100503001A7ADE8EF62E40780060002A3ACE000A70
:08051300B61E3800000076005E
:00000001FF
